Archive member included because of file (symbol)

/home/acer/Andestech/AndeSight133/toolchains/nds32le-elf-V0/libexec/../nds32le-elf/libc/newlib/usr/lib/libc.a(gets.o)
                              hello.o (gets)
/home/acer/Andestech/AndeSight133/toolchains/nds32le-elf-V0/libexec/../nds32le-elf/libc/newlib/usr/lib/libc.a(impure.o)
                              /home/acer/Andestech/AndeSight133/toolchains/nds32le-elf-V0/libexec/../nds32le-elf/libc/newlib/usr/lib/libc.a(gets.o) (_impure_ptr)
/home/acer/Andestech/AndeSight133/toolchains/nds32le-elf-V0/libexec/../nds32le-elf/libc/newlib/usr/lib/libc.a(memcpy.o)
                              cmdui.o (memcpy)
/home/acer/Andestech/AndeSight133/toolchains/nds32le-elf-V0/libexec/../nds32le-elf/libc/newlib/usr/lib/libc.a(printf.o)
                              hello.o (printf)
/home/acer/Andestech/AndeSight133/toolchains/nds32le-elf-V0/libexec/../nds32le-elf/libc/newlib/usr/lib/libc.a(strcmp.o)
                              cmdui.o (strcmp)
/home/acer/Andestech/AndeSight133/toolchains/nds32le-elf-V0/libexec/../nds32le-elf/libc/newlib/usr/lib/libc.a(strcpy.o)
                              cmdui.o (strcpy)
/home/acer/Andestech/AndeSight133/toolchains/nds32le-elf-V0/libexec/../nds32le-elf/libc/newlib/usr/lib/libc.a(strlen.o)
                              cmdui.o (strlen)
/home/acer/Andestech/AndeSight133/toolchains/nds32le-elf-V0/libexec/../nds32le-elf/libc/newlib/usr/lib/libc.a(strncmp.o)
                              cmdui.o (strncmp)
/home/acer/Andestech/AndeSight133/toolchains/nds32le-elf-V0/libexec/../nds32le-elf/libc/newlib/usr/lib/libc.a(strtok.o)
                              cmdui.o (strtok)
/home/acer/Andestech/AndeSight133/toolchains/nds32le-elf-V0/libexec/../nds32le-elf/libc/newlib/usr/lib/libc.a(strtok_r.o)
                              /home/acer/Andestech/AndeSight133/toolchains/nds32le-elf-V0/libexec/../nds32le-elf/libc/newlib/usr/lib/libc.a(strtok.o) (__strtok_r)
/home/acer/Andestech/AndeSight133/toolchains/nds32le-elf-V0/libexec/../nds32le-elf/libc/newlib/usr/lib/libc.a(strtoul.o)
                              cmdui.o (strtoul)
/home/acer/Andestech/AndeSight133/toolchains/nds32le-elf-V0/libexec/../nds32le-elf/libc/newlib/usr/lib/libc.a(vfprintf.o)
                              /home/acer/Andestech/AndeSight133/toolchains/nds32le-elf-V0/libexec/../nds32le-elf/libc/newlib/usr/lib/libc.a(printf.o) (_vfprintf_r)
/home/acer/Andestech/AndeSight133/toolchains/nds32le-elf-V0/libexec/../nds32le-elf/libc/newlib/usr/lib/libc.a(wcrtomb.o)
                              /home/acer/Andestech/AndeSight133/toolchains/nds32le-elf-V0/libexec/../nds32le-elf/libc/newlib/usr/lib/libc.a(vfprintf.o) (_wcrtomb_r)
/home/acer/Andestech/AndeSight133/toolchains/nds32le-elf-V0/libexec/../nds32le-elf/libc/newlib/usr/lib/libc.a(wcsrtombs.o)
                              /home/acer/Andestech/AndeSight133/toolchains/nds32le-elf-V0/libexec/../nds32le-elf/libc/newlib/usr/lib/libc.a(vfprintf.o) (_wcsrtombs_r)
/home/acer/Andestech/AndeSight133/toolchains/nds32le-elf-V0/libexec/../nds32le-elf/libc/newlib/usr/lib/libc.a(wctomb_r.o)
                              /home/acer/Andestech/AndeSight133/toolchains/nds32le-elf-V0/libexec/../nds32le-elf/libc/newlib/usr/lib/libc.a(wcrtomb.o) (_wctomb_r)
/home/acer/Andestech/AndeSight133/toolchains/nds32le-elf-V0/libexec/../nds32le-elf/libc/newlib/usr/lib/libc.a(wsetup.o)
                              /home/acer/Andestech/AndeSight133/toolchains/nds32le-elf-V0/libexec/../nds32le-elf/libc/newlib/usr/lib/libc.a(vfprintf.o) (__swsetup)
/home/acer/Andestech/AndeSight133/toolchains/nds32le-elf-V0/libexec/../nds32le-elf/libc/newlib/usr/lib/libc.a(ctype_.o)
                              /home/acer/Andestech/AndeSight133/toolchains/nds32le-elf-V0/libexec/../nds32le-elf/libc/newlib/usr/lib/libc.a(strtoul.o) (__ctype_ptr)
/home/acer/Andestech/AndeSight133/toolchains/nds32le-elf-V0/libexec/../nds32le-elf/libc/newlib/usr/lib/libc.a(dtoa.o)
                              /home/acer/Andestech/AndeSight133/toolchains/nds32le-elf-V0/libexec/../nds32le-elf/libc/newlib/usr/lib/libc.a(vfprintf.o) (_dtoa_r)
/home/acer/Andestech/AndeSight133/toolchains/nds32le-elf-V0/libexec/../nds32le-elf/libc/newlib/usr/lib/libc.a(fflush.o)
                              /home/acer/Andestech/AndeSight133/toolchains/nds32le-elf-V0/libexec/../nds32le-elf/libc/newlib/usr/lib/libc.a(vfprintf.o) (fflush)
/home/acer/Andestech/AndeSight133/toolchains/nds32le-elf-V0/libexec/../nds32le-elf/libc/newlib/usr/lib/libc.a(findfp.o)
                              /home/acer/Andestech/AndeSight133/toolchains/nds32le-elf-V0/libexec/../nds32le-elf/libc/newlib/usr/lib/libc.a(vfprintf.o) (__sinit)
/home/acer/Andestech/AndeSight133/toolchains/nds32le-elf-V0/libexec/../nds32le-elf/libc/newlib/usr/lib/libc.a(freer.o)
                              /home/acer/Andestech/AndeSight133/toolchains/nds32le-elf-V0/libexec/../nds32le-elf/libc/newlib/usr/lib/libc.a(vfprintf.o) (_free_r)
/home/acer/Andestech/AndeSight133/toolchains/nds32le-elf-V0/libexec/../nds32le-elf/libc/newlib/usr/lib/libc.a(fvwrite.o)
                              /home/acer/Andestech/AndeSight133/toolchains/nds32le-elf-V0/libexec/../nds32le-elf/libc/newlib/usr/lib/libc.a(vfprintf.o) (__sfvwrite)
/home/acer/Andestech/AndeSight133/toolchains/nds32le-elf-V0/libexec/../nds32le-elf/libc/newlib/usr/lib/libc.a(fwalk.o)
                              /home/acer/Andestech/AndeSight133/toolchains/nds32le-elf-V0/libexec/../nds32le-elf/libc/newlib/usr/lib/libc.a(fflush.o) (_fwalk)
/home/acer/Andestech/AndeSight133/toolchains/nds32le-elf-V0/libexec/../nds32le-elf/libc/newlib/usr/lib/libc.a(getchar.o)
                              /home/acer/Andestech/AndeSight133/toolchains/nds32le-elf-V0/libexec/../nds32le-elf/libc/newlib/usr/lib/libc.a(gets.o) (_getchar_r)
/home/acer/Andestech/AndeSight133/toolchains/nds32le-elf-V0/libexec/../nds32le-elf/libc/newlib/usr/lib/libc.a(locale.o)
                              /home/acer/Andestech/AndeSight133/toolchains/nds32le-elf-V0/libexec/../nds32le-elf/libc/newlib/usr/lib/libc.a(wctomb_r.o) (__lc_ctype)
/home/acer/Andestech/AndeSight133/toolchains/nds32le-elf-V0/libexec/../nds32le-elf/libc/newlib/usr/lib/libc.a(makebuf.o)
                              /home/acer/Andestech/AndeSight133/toolchains/nds32le-elf-V0/libexec/../nds32le-elf/libc/newlib/usr/lib/libc.a(wsetup.o) (__smakebuf)
/home/acer/Andestech/AndeSight133/toolchains/nds32le-elf-V0/libexec/../nds32le-elf/libc/newlib/usr/lib/libc.a(mallocr.o)
                              /home/acer/Andestech/AndeSight133/toolchains/nds32le-elf-V0/libexec/../nds32le-elf/libc/newlib/usr/lib/libc.a(freer.o) (__malloc_current_mallinfo)
/home/acer/Andestech/AndeSight133/toolchains/nds32le-elf-V0/libexec/../nds32le-elf/libc/newlib/usr/lib/libc.a(memchr.o)
                              /home/acer/Andestech/AndeSight133/toolchains/nds32le-elf-V0/libexec/../nds32le-elf/libc/newlib/usr/lib/libc.a(vfprintf.o) (memchr)
/home/acer/Andestech/AndeSight133/toolchains/nds32le-elf-V0/libexec/../nds32le-elf/libc/newlib/usr/lib/libc.a(memmove.o)
                              /home/acer/Andestech/AndeSight133/toolchains/nds32le-elf-V0/libexec/../nds32le-elf/libc/newlib/usr/lib/libc.a(fvwrite.o) (memmove)
/home/acer/Andestech/AndeSight133/toolchains/nds32le-elf-V0/libexec/../nds32le-elf/libc/newlib/usr/lib/libc.a(memset.o)
                              /home/acer/Andestech/AndeSight133/toolchains/nds32le-elf-V0/libexec/../nds32le-elf/libc/newlib/usr/lib/libc.a(vfprintf.o) (memset)
/home/acer/Andestech/AndeSight133/toolchains/nds32le-elf-V0/libexec/../nds32le-elf/libc/newlib/usr/lib/libc.a(mlock.o)
                              /home/acer/Andestech/AndeSight133/toolchains/nds32le-elf-V0/libexec/../nds32le-elf/libc/newlib/usr/lib/libc.a(freer.o) (__malloc_lock)
/home/acer/Andestech/AndeSight133/toolchains/nds32le-elf-V0/libexec/../nds32le-elf/libc/newlib/usr/lib/libc.a(mprec.o)
                              /home/acer/Andestech/AndeSight133/toolchains/nds32le-elf-V0/libexec/../nds32le-elf/libc/newlib/usr/lib/libc.a(dtoa.o) (__mprec_bigtens)
/home/acer/Andestech/AndeSight133/toolchains/nds32le-elf-V0/libexec/../nds32le-elf/libc/newlib/usr/lib/libc.a(reallocr.o)
                              /home/acer/Andestech/AndeSight133/toolchains/nds32le-elf-V0/libexec/../nds32le-elf/libc/newlib/usr/lib/libc.a(fvwrite.o) (_realloc_r)
/home/acer/Andestech/AndeSight133/toolchains/nds32le-elf-V0/libexec/../nds32le-elf/libc/newlib/usr/lib/libc.a(rget.o)
                              /home/acer/Andestech/AndeSight133/toolchains/nds32le-elf-V0/libexec/../nds32le-elf/libc/newlib/usr/lib/libc.a(getchar.o) (__srget)
/home/acer/Andestech/AndeSight133/toolchains/nds32le-elf-V0/libexec/../nds32le-elf/libc/newlib/usr/lib/libc.a(s_isinf.o)
                              /home/acer/Andestech/AndeSight133/toolchains/nds32le-elf-V0/libexec/../nds32le-elf/libc/newlib/usr/lib/libc.a(vfprintf.o) (isinf)
/home/acer/Andestech/AndeSight133/toolchains/nds32le-elf-V0/libexec/../nds32le-elf/libc/newlib/usr/lib/libc.a(s_isnan.o)
                              /home/acer/Andestech/AndeSight133/toolchains/nds32le-elf-V0/libexec/../nds32le-elf/libc/newlib/usr/lib/libc.a(vfprintf.o) (isnan)
/home/acer/Andestech/AndeSight133/toolchains/nds32le-elf-V0/libexec/../nds32le-elf/libc/newlib/usr/lib/libc.a(sbrkr.o)
                              /home/acer/Andestech/AndeSight133/toolchains/nds32le-elf-V0/libexec/../nds32le-elf/libc/newlib/usr/lib/libc.a(freer.o) (_sbrk_r)
/home/acer/Andestech/AndeSight133/toolchains/nds32le-elf-V0/libexec/../nds32le-elf/libc/newlib/usr/lib/libc.a(stdio.o)
                              /home/acer/Andestech/AndeSight133/toolchains/nds32le-elf-V0/libexec/../nds32le-elf/libc/newlib/usr/lib/libc.a(findfp.o) (__sread)
/home/acer/Andestech/AndeSight133/toolchains/nds32le-elf-V0/libexec/../nds32le-elf/libc/newlib/usr/lib/libc.a(syssbrk.o)
                              /home/acer/Andestech/AndeSight133/toolchains/nds32le-elf-V0/libexec/../nds32le-elf/libc/newlib/usr/lib/libc.a(sbrkr.o) (sbrk)
/home/acer/Andestech/AndeSight133/toolchains/nds32le-elf-V0/libexec/../nds32le-elf/libc/newlib/usr/lib/libc.a(writer.o)
                              /home/acer/Andestech/AndeSight133/toolchains/nds32le-elf-V0/libexec/../nds32le-elf/libc/newlib/usr/lib/libc.a(stdio.o) (_write_r)
/home/acer/Andestech/AndeSight133/toolchains/nds32le-elf-V0/libexec/../nds32le-elf/libc/newlib/usr/lib/libc.a(callocr.o)
                              /home/acer/Andestech/AndeSight133/toolchains/nds32le-elf-V0/libexec/../nds32le-elf/libc/newlib/usr/lib/libc.a(mprec.o) (_calloc_r)
/home/acer/Andestech/AndeSight133/toolchains/nds32le-elf-V0/libexec/../nds32le-elf/libc/newlib/usr/lib/libc.a(closer.o)
                              /home/acer/Andestech/AndeSight133/toolchains/nds32le-elf-V0/libexec/../nds32le-elf/libc/newlib/usr/lib/libc.a(stdio.o) (_close_r)
/home/acer/Andestech/AndeSight133/toolchains/nds32le-elf-V0/libexec/../nds32le-elf/libc/newlib/usr/lib/libc.a(fclose.o)
                              /home/acer/Andestech/AndeSight133/toolchains/nds32le-elf-V0/libexec/../nds32le-elf/libc/newlib/usr/lib/libc.a(findfp.o) (fclose)
/home/acer/Andestech/AndeSight133/toolchains/nds32le-elf-V0/libexec/../nds32le-elf/libc/newlib/usr/lib/libc.a(fstatr.o)
                              /home/acer/Andestech/AndeSight133/toolchains/nds32le-elf-V0/libexec/../nds32le-elf/libc/newlib/usr/lib/libc.a(makebuf.o) (_fstat_r)
/home/acer/Andestech/AndeSight133/toolchains/nds32le-elf-V0/libexec/../nds32le-elf/libc/newlib/usr/lib/libc.a(lseekr.o)
                              /home/acer/Andestech/AndeSight133/toolchains/nds32le-elf-V0/libexec/../nds32le-elf/libc/newlib/usr/lib/libc.a(stdio.o) (_lseek_r)
/home/acer/Andestech/AndeSight133/toolchains/nds32le-elf-V0/libexec/../nds32le-elf/libc/newlib/usr/lib/libc.a(readr.o)
                              /home/acer/Andestech/AndeSight133/toolchains/nds32le-elf-V0/libexec/../nds32le-elf/libc/newlib/usr/lib/libc.a(stdio.o) (_read_r)
/home/acer/Andestech/AndeSight133/toolchains/nds32le-elf-V0/libexec/../nds32le-elf/libc/newlib/usr/lib/libc.a(reent.o)
                              /home/acer/Andestech/AndeSight133/toolchains/nds32le-elf-V0/libexec/../nds32le-elf/libc/newlib/usr/lib/libc.a(sbrkr.o) (errno)
/home/acer/Andestech/AndeSight133/toolchains/nds32le-elf-V0/libexec/../nds32le-elf/libc/newlib/usr/lib/libc.a(refill.o)
                              /home/acer/Andestech/AndeSight133/toolchains/nds32le-elf-V0/libexec/../nds32le-elf/libc/newlib/usr/lib/libc.a(rget.o) (__srefill)
/home/acer/Andestech/AndeSight133/toolchains/nds32le-elf-V0/libexec/../nds32le-elf/libc/newlib/usr/lib/libc.a(sysclose.o)
                              /home/acer/Andestech/AndeSight133/toolchains/nds32le-elf-V0/libexec/../nds32le-elf/libc/newlib/usr/lib/libc.a(closer.o) (close)
/home/acer/Andestech/AndeSight133/toolchains/nds32le-elf-V0/libexec/../nds32le-elf/libc/newlib/usr/lib/libc.a(sysfstat.o)
                              /home/acer/Andestech/AndeSight133/toolchains/nds32le-elf-V0/libexec/../nds32le-elf/libc/newlib/usr/lib/libc.a(fstatr.o) (fstat)
/home/acer/Andestech/AndeSight133/toolchains/nds32le-elf-V0/libexec/../nds32le-elf/libc/newlib/usr/lib/libc.a(syslseek.o)
                              /home/acer/Andestech/AndeSight133/toolchains/nds32le-elf-V0/libexec/../nds32le-elf/libc/newlib/usr/lib/libc.a(lseekr.o) (lseek)
/home/acer/Andestech/AndeSight133/toolchains/nds32le-elf-V0/libexec/../nds32le-elf/libc/newlib/usr/lib/libc.a(sysread.o)
                              /home/acer/Andestech/AndeSight133/toolchains/nds32le-elf-V0/libexec/../nds32le-elf/libc/newlib/usr/lib/libc.a(readr.o) (read)
/home/acer/Andestech/AndeSight133/toolchains/nds32le-elf-V0/libexec/../nds32le-elf/libc/newlib/usr/lib/libc.a(syswrite.o)
                              /home/acer/Andestech/AndeSight133/toolchains/nds32le-elf-V0/libexec/../nds32le-elf/libc/newlib/usr/lib/libc.a(writer.o) (write)
/home/acer/Andestech/AndeSight133/toolchains/nds32le-elf-V0/libexec/../lib/gcc/nds32le-elf/3.4.4/static/newlib/libgcc.a(_udivsi3.o)
                              /home/acer/Andestech/AndeSight133/toolchains/nds32le-elf-V0/libexec/../nds32le-elf/libc/newlib/usr/lib/libc.a(strtoul.o) (__udivsi3)
/home/acer/Andestech/AndeSight133/toolchains/nds32le-elf-V0/libexec/../lib/gcc/nds32le-elf/3.4.4/static/newlib/libgcc.a(_umodsi3.o)
                              /home/acer/Andestech/AndeSight133/toolchains/nds32le-elf-V0/libexec/../nds32le-elf/libc/newlib/usr/lib/libc.a(strtoul.o) (__umodsi3)
/home/acer/Andestech/AndeSight133/toolchains/nds32le-elf-V0/libexec/../lib/gcc/nds32le-elf/3.4.4/static/newlib/libgcc.a(lib1csrc.o)
                              /home/acer/Andestech/AndeSight133/toolchains/nds32le-elf-V0/libexec/../nds32le-elf/libc/newlib/usr/lib/libc.a(dtoa.o) (__floatsidf)
/home/acer/Andestech/AndeSight133/toolchains/nds32le-elf-V0/libexec/../lib/gcc/nds32le-elf/3.4.4/static/newlib/libgcc.a(_negdi2.o)
                              /home/acer/Andestech/AndeSight133/toolchains/nds32le-elf-V0/libexec/../nds32le-elf/libc/newlib/usr/lib/libc.a(vfprintf.o) (__negdi2)
/home/acer/Andestech/AndeSight133/toolchains/nds32le-elf-V0/libexec/../lib/gcc/nds32le-elf/3.4.4/static/newlib/libgcc.a(_udivdi3.o)
                              /home/acer/Andestech/AndeSight133/toolchains/nds32le-elf-V0/libexec/../nds32le-elf/libc/newlib/usr/lib/libc.a(vfprintf.o) (__udivdi3)
/home/acer/Andestech/AndeSight133/toolchains/nds32le-elf-V0/libexec/../lib/gcc/nds32le-elf/3.4.4/static/newlib/libgcc.a(_umoddi3.o)
                              /home/acer/Andestech/AndeSight133/toolchains/nds32le-elf-V0/libexec/../nds32le-elf/libc/newlib/usr/lib/libc.a(vfprintf.o) (__umoddi3)
/home/acer/Andestech/AndeSight133/toolchains/nds32le-elf-V0/libexec/../lib/gcc/nds32le-elf/3.4.4/static/newlib/libgcc.a(_eq_df.o)
                              /home/acer/Andestech/AndeSight133/toolchains/nds32le-elf-V0/libexec/../nds32le-elf/libc/newlib/usr/lib/libc.a(vfprintf.o) (__eqdf2)
/home/acer/Andestech/AndeSight133/toolchains/nds32le-elf-V0/libexec/../lib/gcc/nds32le-elf/3.4.4/static/newlib/libgcc.a(_ne_df.o)
                              /home/acer/Andestech/AndeSight133/toolchains/nds32le-elf-V0/libexec/../nds32le-elf/libc/newlib/usr/lib/libc.a(vfprintf.o) (__nedf2)
/home/acer/Andestech/AndeSight133/toolchains/nds32le-elf-V0/libexec/../lib/gcc/nds32le-elf/3.4.4/static/newlib/libgcc.a(_gt_df.o)
                              /home/acer/Andestech/AndeSight133/toolchains/nds32le-elf-V0/libexec/../nds32le-elf/libc/newlib/usr/lib/libc.a(dtoa.o) (__gtdf2)
/home/acer/Andestech/AndeSight133/toolchains/nds32le-elf-V0/libexec/../lib/gcc/nds32le-elf/3.4.4/static/newlib/libgcc.a(_ge_df.o)
                              /home/acer/Andestech/AndeSight133/toolchains/nds32le-elf-V0/libexec/../nds32le-elf/libc/newlib/usr/lib/libc.a(dtoa.o) (__gedf2)
/home/acer/Andestech/AndeSight133/toolchains/nds32le-elf-V0/libexec/../lib/gcc/nds32le-elf/3.4.4/static/newlib/libgcc.a(_lt_df.o)
                              /home/acer/Andestech/AndeSight133/toolchains/nds32le-elf-V0/libexec/../nds32le-elf/libc/newlib/usr/lib/libc.a(vfprintf.o) (__ltdf2)
/home/acer/Andestech/AndeSight133/toolchains/nds32le-elf-V0/libexec/../lib/gcc/nds32le-elf/3.4.4/static/newlib/libgcc.a(_clz.o)
                              /home/acer/Andestech/AndeSight133/toolchains/nds32le-elf-V0/libexec/../lib/gcc/nds32le-elf/3.4.4/static/newlib/libgcc.a(_udivdi3.o) (__clz_tab)
/home/acer/Andestech/AndeSight133/toolchains/nds32le-elf-V0/libexec/../lib/gcc/nds32le-elf/3.4.4/static/newlib/libgcc.a(_unpack_df.o)
                              /home/acer/Andestech/AndeSight133/toolchains/nds32le-elf-V0/libexec/../lib/gcc/nds32le-elf/3.4.4/static/newlib/libgcc.a(_eq_df.o) (__unpack_d)
/home/acer/Andestech/AndeSight133/toolchains/nds32le-elf-V0/libexec/../lib/gcc/nds32le-elf/3.4.4/static/newlib/libgcc.a(_fpcmp_parts_df.o)
                              /home/acer/Andestech/AndeSight133/toolchains/nds32le-elf-V0/libexec/../lib/gcc/nds32le-elf/3.4.4/static/newlib/libgcc.a(_eq_df.o) (__fpcmp_parts_d)
/home/acer/Andestech/AndeSight133/toolchains/nds32le-elf-V0/libexec/../nds32le-elf/libc/newlib/usr/lib/libgloss.a(syscalls.o)
                              /home/acer/Andestech/AndeSight133/toolchains/nds32le-elf-V0/libexec/../nds32le-elf/libc/newlib/usr/lib/libc.a(syssbrk.o) (_sbrk)

Allocating common symbols
Common symbol       size              file

UserSymbolTable     0x2100            cmdui.o

Memory Configuration

Name             Origin             Length             Attributes
*default*        0x00000000         0xffffffff

Linker script and memory map

START GROUP
LOAD hello.o
LOAD ssp.o
LOAD cmdui.o
LOAD interrupt.o
LOAD irq.o
LOAD fiq.o
LOAD boot.o
END GROUP
                0x00500000                PROVIDE (__executable_start, 0x500000)
                0x00500000                . = 0x500000

.interp
 *(.interp)

.hash
 *(.hash)

.dynsym
 *(.dynsym)

.dynstr
 *(.dynstr)

.gnu.version
 *(.gnu.version)

.gnu.version_d
 *(.gnu.version_d)

.gnu.version_r
 *(.gnu.version_r)

.rel.init
 *(.rel.init)

.rela.init
 *(.rela.init)

.rel.text
 *(.rel.text .rel.text.* .rel.gnu.linkonce.t.*)

.rela.text      0x00500000        0x0
 *(.rela.text .rela.text.* .rela.gnu.linkonce.t.*)

.rel.fini
 *(.rel.fini)

.rela.fini
 *(.rela.fini)

.rel.rodata
 *(.rel.rodata .rel.rodata.* .rel.gnu.linkonce.r.*)

.rela.rodata
 *(.rela.rodata .rela.rodata.* .rela.gnu.linkonce.r.*)

.rel.data.rel.ro
 *(.rel.data.rel.ro*)

.rela.data.rel.ro
 *(.rel.data.rel.ro*)

.rel.data
 *(.rel.data .rel.data.* .rel.gnu.linkonce.d.*)

.rela.data
 *(.rela.data .rela.data.* .rela.gnu.linkonce.d.*)

.rel.tdata
 *(.rel.tdata .rel.tdata.* .rel.gnu.linkonce.td.*)

.rela.tdata
 *(.rela.tdata .rela.tdata.* .rela.gnu.linkonce.td.*)

.rel.tbss
 *(.rel.tbss .rel.tbss.* .rel.gnu.linkonce.tb.*)

.rela.tbss
 *(.rela.tbss .rela.tbss.* .rela.gnu.linkonce.tb.*)

.rel.ctors
 *(.rel.ctors)

.rela.ctors
 *(.rela.ctors)

.rel.dtors
 *(.rel.dtors)

.rela.dtors
 *(.rela.dtors)

.rel.got
 *(.rel.got)

.rela.got
 *(.rela.got)

.rel.sdata
 *(.rel.sdata .rel.sdata.* .rel.gnu.linkonce.s.*)

.rela.sdata
 *(.rela.sdata .rela.sdata.* .rela.gnu.linkonce.s.*)

.rel.sbss
 *(.rel.sbss .rel.sbss.* .rel.gnu.linkonce.sb.*)

.rela.sbss
 *(.rela.sbss .rela.sbss.* .rela.gnu.linkonce.sb.*)

.rel.sdata2
 *(.rel.sdata2 .rel.sdata2.* .rel.gnu.linkonce.s2.*)

.rela.sdata2
 *(.rela.sdata2 .rela.sdata2.* .rela.gnu.linkonce.s2.*)

.rel.sbss2
 *(.rel.sbss2 .rel.sbss2.* .rel.gnu.linkonce.sb2.*)

.rela.sbss2
 *(.rela.sbss2 .rela.sbss2.* .rela.gnu.linkonce.sb2.*)

.rel.bss
 *(.rel.bss .rel.bss.* .rel.gnu.linkonce.b.*)

.rela.bss
 *(.rela.bss .rela.bss.* .rela.gnu.linkonce.b.*)

.rel.plt
 *(.rel.plt)

.rela.plt
 *(.rela.plt)

.text           0x00500000     0xdb80
 *(.text .stub .text.* .gnu.linkonce.t.*)
 .text          0x00500000      0x5ec hello.o
                0x005003ec                PlayCmd
                0x00500000                main
                0x00500178                RecordCmd
 .text          0x005005ec      0x5d0 ssp.o
                0x005009c4                fLib_AC97_WriteData
                0x00500914                fLib_SSP_GetTxFIFOLen
                0x005005ec                fLib_SetSSPFrame
                0x00500a98                fLib_ReturnTxFIFO_Count
                0x00500af8                fLib_AC97_WriteRegisterEx
                0x00500978                fLib_AC97_SetSlotValidReg
                0x0050066c                fLib_SSPClearTxFIFO
                0x005007e4                fLib_SetSSP_Enable
                0x00500880                fLib_SetSSP_IntMask
                0x00500764                fLib_SetSSP_ColdReset
                0x005006e8                fLib_SSPClearRxFIFO
 .text          0x00500bbc     0x1d08 cmdui.o
                0x005023bc                FindOption
                0x0050207c                SaveArgument
                0x00501334                WriteUserSymbol
                0x005017e0                IsDigit
                0x005018e4                ParameterIsConstant
                0x005010bc                ParseCommand
                0x005013ac                ParameterIsUserSymbol
                0x00501640                ParameterIsArithmeticOperation
                0x00500cec                fLib_InitUserSymbol
                0x005014a0                ParameterIsLogicalOperation
                0x00502528                FreeCmdArgumentOption
                0x00501bec                ParameterToNumber
                0x00501cb0                ParseCommandParameter
                0x00501248                NewUserSymbol
                0x0050247c                FineSubOption
                0x00502718                HelpCmd
                0x00500bbc                fLib_InsertCommand
                0x00501a54                ParameterIsMemory
                0x00500dec                fLib_ExecuteCommand
                0x005011fc                IsCommandBreak
                0x00501838                IsXDigit
 .text          0x005028c4      0x15c interrupt.o
                0x0050296c                fLib_EnableInt
                0x005028c4                fLib_DisableInt
 .text          0x00502a20       0xa4 irq.o
                0x00502a20                MaskIRQ
                0x00502a74                UnmaskIRQ
 .text          0x00502ac4       0xa4 fiq.o
                0x00502b18                UnmaskFIQ
                0x00502ac4                MaskFIQ
 .text          0x00502b68       0x40 boot.o
                0x00502b88                EnableIRQ
                0x00502b68                EnableFIQ
 .text          0x00502ba8       0x8c /home/acer/Andestech/AndeSight133/toolchains/nds32le-elf-V0/libexec/../nds32le-elf/libc/newlib/usr/lib/libc.a(gets.o)
                0x00502c08                gets
                0x00502ba8                _gets_r
 .text          0x00502c34       0x68 /home/acer/Andestech/AndeSight133/toolchains/nds32le-elf-V0/libexec/../nds32le-elf/libc/newlib/usr/lib/libc.a(memcpy.o)
                0x00502c34                memcpy
 .text          0x00502c9c       0x80 /home/acer/Andestech/AndeSight133/toolchains/nds32le-elf-V0/libexec/../nds32le-elf/libc/newlib/usr/lib/libc.a(printf.o)
                0x00502cd8                printf
                0x00502c9c                _printf_r
 .text          0x00502d1c       0x84 /home/acer/Andestech/AndeSight133/toolchains/nds32le-elf-V0/libexec/../nds32le-elf/libc/newlib/usr/lib/libc.a(strcmp.o)
                0x00502d1c                strcmp
 .text          0x00502da0       0x80 /home/acer/Andestech/AndeSight133/toolchains/nds32le-elf-V0/libexec/../nds32le-elf/libc/newlib/usr/lib/libc.a(strcpy.o)
                0x00502da0                strcpy
 .text          0x00502e20       0x7c /home/acer/Andestech/AndeSight133/toolchains/nds32le-elf-V0/libexec/../nds32le-elf/libc/newlib/usr/lib/libc.a(strlen.o)
                0x00502e20                strlen
 .text          0x00502e9c       0xb4 /home/acer/Andestech/AndeSight133/toolchains/nds32le-elf-V0/libexec/../nds32le-elf/libc/newlib/usr/lib/libc.a(strncmp.o)
                0x00502e9c                strncmp
 .text          0x00502f50       0x30 /home/acer/Andestech/AndeSight133/toolchains/nds32le-elf-V0/libexec/../nds32le-elf/libc/newlib/usr/lib/libc.a(strtok.o)
                0x00502f50                strtok
 .text          0x00502f80       0xbc /home/acer/Andestech/AndeSight133/toolchains/nds32le-elf-V0/libexec/../nds32le-elf/libc/newlib/usr/lib/libc.a(strtok_r.o)
                0x00503018                strtok_r
                0x00502f80                __strtok_r
 .text          0x0050303c      0x1d0 /home/acer/Andestech/AndeSight133/toolchains/nds32le-elf-V0/libexec/../nds32le-elf/libc/newlib/usr/lib/libc.a(strtoul.o)
                0x005031d8                strtoul
                0x0050303c                _strtoul_r
 .text          0x0050320c     0x1b8c /home/acer/Andestech/AndeSight133/toolchains/nds32le-elf-V0/libexec/../nds32le-elf/libc/newlib/usr/lib/libc.a(vfprintf.o)
                0x00503250                _vfprintf_r
                0x00504d64                vfprintf
 .text          0x00504d98       0x88 /home/acer/Andestech/AndeSight133/toolchains/nds32le-elf-V0/libexec/../nds32le-elf/libc/newlib/usr/lib/libc.a(wcrtomb.o)
                0x00504d98                _wcrtomb_r
                0x00504dec                wcrtomb
 .text          0x00504e20      0x100 /home/acer/Andestech/AndeSight133/toolchains/nds32le-elf-V0/libexec/../nds32le-elf/libc/newlib/usr/lib/libc.a(wcsrtombs.o)
                0x00504e20                _wcsrtombs_r
                0x00504ee8                wcsrtombs
 .text          0x00504f20      0x390 /home/acer/Andestech/AndeSight133/toolchains/nds32le-elf-V0/libexec/../nds32le-elf/libc/newlib/usr/lib/libc.a(wctomb_r.o)
                0x00504f20                _wctomb_r
 .text          0x005052b0       0xec /home/acer/Andestech/AndeSight133/toolchains/nds32le-elf-V0/libexec/../nds32le-elf/libc/newlib/usr/lib/libc.a(wsetup.o)
                0x005052b0                __swsetup
 .text          0x0050539c     0x1348 /home/acer/Andestech/AndeSight133/toolchains/nds32le-elf-V0/libexec/../nds32le-elf/libc/newlib/usr/lib/libc.a(dtoa.o)
                0x00505514                _dtoa_r
 .text          0x005066e4       0xd0 /home/acer/Andestech/AndeSight133/toolchains/nds32le-elf-V0/libexec/../nds32le-elf/libc/newlib/usr/lib/libc.a(fflush.o)
                0x005066e4                fflush
 .text          0x005067b4      0x340 /home/acer/Andestech/AndeSight133/toolchains/nds32le-elf-V0/libexec/../nds32le-elf/libc/newlib/usr/lib/libc.a(findfp.o)
                0x00506924                __sinit
                0x00506810                __sfmoreglue
                0x005068cc                _cleanup
                0x005068a4                _cleanup_r
                0x00506a94                __fp_lock_all
                0x00506874                __sfp_lock_acquire
                0x005069ac                __sfp
                0x0050690c                __sinit_lock_release
                0x00506ac4                __fp_unlock_all
                0x0050688c                __sfp_lock_release
                0x005068f4                __sinit_lock_acquire
 .text          0x00506af4      0x368 /home/acer/Andestech/AndeSight133/toolchains/nds32le-elf-V0/libexec/../nds32le-elf/libc/newlib/usr/lib/libc.a(freer.o)
                0x00506bec                _free_r
                0x00506af4                _malloc_trim_r
 .text          0x00506e5c      0x380 /home/acer/Andestech/AndeSight133/toolchains/nds32le-elf-V0/libexec/../nds32le-elf/libc/newlib/usr/lib/libc.a(fvwrite.o)
                0x00506e5c                __sfvwrite
 .text          0x005071dc      0x118 /home/acer/Andestech/AndeSight133/toolchains/nds32le-elf-V0/libexec/../nds32le-elf/libc/newlib/usr/lib/libc.a(fwalk.o)
                0x005071dc                _fwalk
                0x00507264                _fwalk_reent
 .text          0x005072f4       0x6c /home/acer/Andestech/AndeSight133/toolchains/nds32le-elf-V0/libexec/../nds32le-elf/libc/newlib/usr/lib/libc.a(getchar.o)
                0x00507338                getchar
                0x005072f4                _getchar_r
 .text          0x00507360      0x10c /home/acer/Andestech/AndeSight133/toolchains/nds32le-elf-V0/libexec/../nds32le-elf/libc/newlib/usr/lib/libc.a(locale.o)
                0x00507360                _setlocale_r
                0x005073d4                __locale_charset
                0x005073f4                _localeconv_r
                0x00507414                setlocale
                0x00507444                localeconv
 .text          0x0050746c      0x138 /home/acer/Andestech/AndeSight133/toolchains/nds32le-elf-V0/libexec/../nds32le-elf/libc/newlib/usr/lib/libc.a(makebuf.o)
                0x0050746c                __smakebuf
 .text          0x005075a4      0x68c /home/acer/Andestech/AndeSight133/toolchains/nds32le-elf-V0/libexec/../nds32le-elf/libc/newlib/usr/lib/libc.a(mallocr.o)
                0x005075a4                _malloc_r
 .text          0x00507c30       0xa0 /home/acer/Andestech/AndeSight133/toolchains/nds32le-elf-V0/libexec/../nds32le-elf/libc/newlib/usr/lib/libc.a(memchr.o)
                0x00507c30                memchr
 .text          0x00507cd0       0x94 /home/acer/Andestech/AndeSight133/toolchains/nds32le-elf-V0/libexec/../nds32le-elf/libc/newlib/usr/lib/libc.a(memmove.o)
                0x00507cd0                memmove
 .text          0x00507d64       0x6c /home/acer/Andestech/AndeSight133/toolchains/nds32le-elf-V0/libexec/../nds32le-elf/libc/newlib/usr/lib/libc.a(memset.o)
                0x00507d64                memset
 .text          0x00507dd0       0x30 /home/acer/Andestech/AndeSight133/toolchains/nds32le-elf-V0/libexec/../nds32le-elf/libc/newlib/usr/lib/libc.a(mlock.o)
                0x00507de8                __malloc_unlock
                0x00507dd0                __malloc_lock
 .text          0x00507e00      0xbb0 /home/acer/Andestech/AndeSight133/toolchains/nds32le-elf-V0/libexec/../nds32le-elf/libc/newlib/usr/lib/libc.a(mprec.o)
                0x00508940                _mprec_log10
                0x00508048                _hi0bits
                0x00507e00                _Balloc
                0x00508790                _d2b
                0x00508178                _multiply
                0x005088b4                _ratio
                0x00507f80                _s2b
                0x00508140                _i2b
                0x005080bc                _lo0bits
                0x005084b0                __mcmp
                0x005082ec                _pow5mult
                0x0050865c                _ulp
                0x005086c0                _b2d
                0x00507eb4                _multadd
                0x00508510                __mdiff
                0x005083e4                _lshift
                0x00507e88                _Bfree
 .text          0x005089b0      0x408 /home/acer/Andestech/AndeSight133/toolchains/nds32le-elf-V0/libexec/../nds32le-elf/libc/newlib/usr/lib/libc.a(reallocr.o)
                0x005089b0                _realloc_r
 .text          0x00508db8       0x44 /home/acer/Andestech/AndeSight133/toolchains/nds32le-elf-V0/libexec/../nds32le-elf/libc/newlib/usr/lib/libc.a(rget.o)
                0x00508db8                __srget
 .text          0x00508dfc       0x48 /home/acer/Andestech/AndeSight133/toolchains/nds32le-elf-V0/libexec/../nds32le-elf/libc/newlib/usr/lib/libc.a(s_isinf.o)
                0x00508dfc                isinf
 .text          0x00508e44       0x3c /home/acer/Andestech/AndeSight133/toolchains/nds32le-elf-V0/libexec/../nds32le-elf/libc/newlib/usr/lib/libc.a(s_isnan.o)
                0x00508e44                isnan
 .text          0x00508e80       0x48 /home/acer/Andestech/AndeSight133/toolchains/nds32le-elf-V0/libexec/../nds32le-elf/libc/newlib/usr/lib/libc.a(sbrkr.o)
                0x00508e80                _sbrk_r
 .text          0x00508ec8      0x190 /home/acer/Andestech/AndeSight133/toolchains/nds32le-elf-V0/libexec/../nds32le-elf/libc/newlib/usr/lib/libc.a(stdio.o)
                0x00508fc8                __sseek
                0x00508ec8                __sread
                0x0050902c                __sclose
                0x00508f28                __swrite
 .text          0x00509058       0x20 /home/acer/Andestech/AndeSight133/toolchains/nds32le-elf-V0/libexec/../nds32le-elf/libc/newlib/usr/lib/libc.a(syssbrk.o)
                0x00509058                sbrk
 .text          0x00509078       0x4c /home/acer/Andestech/AndeSight133/toolchains/nds32le-elf-V0/libexec/../nds32le-elf/libc/newlib/usr/lib/libc.a(writer.o)
                0x00509078                _write_r
 .text          0x005090c4       0x88 /home/acer/Andestech/AndeSight133/toolchains/nds32le-elf-V0/libexec/../nds32le-elf/libc/newlib/usr/lib/libc.a(callocr.o)
                0x005090c4                _calloc_r
 .text          0x0050914c       0x48 /home/acer/Andestech/AndeSight133/toolchains/nds32le-elf-V0/libexec/../nds32le-elf/libc/newlib/usr/lib/libc.a(closer.o)
                0x0050914c                _close_r
 .text          0x00509194      0x14c /home/acer/Andestech/AndeSight133/toolchains/nds32le-elf-V0/libexec/../nds32le-elf/libc/newlib/usr/lib/libc.a(fclose.o)
                0x00509194                _fclose_r
                0x005092b4                fclose
 .text          0x005092e0       0x4c /home/acer/Andestech/AndeSight133/toolchains/nds32le-elf-V0/libexec/../nds32le-elf/libc/newlib/usr/lib/libc.a(fstatr.o)
                0x005092e0                _fstat_r
 .text          0x0050932c       0x4c /home/acer/Andestech/AndeSight133/toolchains/nds32le-elf-V0/libexec/../nds32le-elf/libc/newlib/usr/lib/libc.a(lseekr.o)
                0x0050932c                _lseek_r
 .text          0x00509378       0x4c /home/acer/Andestech/AndeSight133/toolchains/nds32le-elf-V0/libexec/../nds32le-elf/libc/newlib/usr/lib/libc.a(readr.o)
                0x00509378                _read_r
 .text          0x005093c4      0x1d0 /home/acer/Andestech/AndeSight133/toolchains/nds32le-elf-V0/libexec/../nds32le-elf/libc/newlib/usr/lib/libc.a(reent.o)
                0x005093c4                cleanup_glue
                0x00509428                _reclaim_reent
                0x0050951c                _wrapup_reent
 .text          0x00509594      0x1a4 /home/acer/Andestech/AndeSight133/toolchains/nds32le-elf-V0/libexec/../nds32le-elf/libc/newlib/usr/lib/libc.a(refill.o)
                0x005095d0                __srefill
 .text          0x00509738       0x20 /home/acer/Andestech/AndeSight133/toolchains/nds32le-elf-V0/libexec/../nds32le-elf/libc/newlib/usr/lib/libc.a(sysclose.o)
                0x00509738                close
 .text          0x00509758       0x20 /home/acer/Andestech/AndeSight133/toolchains/nds32le-elf-V0/libexec/../nds32le-elf/libc/newlib/usr/lib/libc.a(sysfstat.o)
                0x00509758                fstat
 .text          0x00509778       0x20 /home/acer/Andestech/AndeSight133/toolchains/nds32le-elf-V0/libexec/../nds32le-elf/libc/newlib/usr/lib/libc.a(syslseek.o)
                0x00509778                lseek
 .text          0x00509798       0x20 /home/acer/Andestech/AndeSight133/toolchains/nds32le-elf-V0/libexec/../nds32le-elf/libc/newlib/usr/lib/libc.a(sysread.o)
                0x00509798                read
 .text          0x005097b8       0x20 /home/acer/Andestech/AndeSight133/toolchains/nds32le-elf-V0/libexec/../nds32le-elf/libc/newlib/usr/lib/libc.a(syswrite.o)
                0x005097b8                write
 .text          0x005097d8       0x40 /home/acer/Andestech/AndeSight133/toolchains/nds32le-elf-V0/libexec/../lib/gcc/nds32le-elf/3.4.4/static/newlib/libgcc.a(_udivsi3.o)
                0x005097d8                __udivsi3
 .text          0x00509818       0x3c /home/acer/Andestech/AndeSight133/toolchains/nds32le-elf-V0/libexec/../lib/gcc/nds32le-elf/3.4.4/static/newlib/libgcc.a(_umodsi3.o)
                0x00509818                __umodsi3
 .text          0x00509854     0x2f70 /home/acer/Andestech/AndeSight133/toolchains/nds32le-elf-V0/libexec/../lib/gcc/nds32le-elf/3.4.4/static/newlib/libgcc.a(lib1csrc.o)
                0x0050acf4                __divsf3
                0x0050a47c                __fixsfsi
                0x0050ab18                __subsf3
                0x00509a18                float32_is_signaling_nan
                0x0050a354                __floatsidf
                0x005099f8                float32_is_nan
                0x0050a554                __extendsfdf2
                0x0050bbd4                __adddf3
                0x00509b14                float64_is_nan
                0x0050af08                __fixdfsi
                0x005099d0                float_raise
                0x0050a310                __floatsisf
                0x0050c1c0                __divdf3
                0x00509b58                float64_is_signaling_nan
                0x0050bd2c                __muldf3
                0x0050b074                __truncdfsf2
                0x0050ab54                __mulsf3
                0x0050bc80                __subdf3
                0x0050aadc                __addsf3
 .text          0x0050c7c4       0x28 /home/acer/Andestech/AndeSight133/toolchains/nds32le-elf-V0/libexec/../lib/gcc/nds32le-elf/3.4.4/static/newlib/libgcc.a(_negdi2.o)
                0x0050c7c4                __negdi2
 .text          0x0050c7ec      0x528 /home/acer/Andestech/AndeSight133/toolchains/nds32le-elf-V0/libexec/../lib/gcc/nds32le-elf/3.4.4/static/newlib/libgcc.a(_udivdi3.o)
                0x0050c7ec                __udivdi3
 .text          0x0050cd14      0x5c4 /home/acer/Andestech/AndeSight133/toolchains/nds32le-elf-V0/libexec/../lib/gcc/nds32le-elf/3.4.4/static/newlib/libgcc.a(_umoddi3.o)
                0x0050cd14                __umoddi3
 .text          0x0050d2d8       0xa0 /home/acer/Andestech/AndeSight133/toolchains/nds32le-elf-V0/libexec/../lib/gcc/nds32le-elf/3.4.4/static/newlib/libgcc.a(_eq_df.o)
                0x0050d2f4                __eqdf2
 .text          0x0050d378       0xa0 /home/acer/Andestech/AndeSight133/toolchains/nds32le-elf-V0/libexec/../lib/gcc/nds32le-elf/3.4.4/static/newlib/libgcc.a(_ne_df.o)
                0x0050d394                __nedf2
 .text          0x0050d418       0xa0 /home/acer/Andestech/AndeSight133/toolchains/nds32le-elf-V0/libexec/../lib/gcc/nds32le-elf/3.4.4/static/newlib/libgcc.a(_gt_df.o)
                0x0050d434                __gtdf2
 .text          0x0050d4b8       0xa0 /home/acer/Andestech/AndeSight133/toolchains/nds32le-elf-V0/libexec/../lib/gcc/nds32le-elf/3.4.4/static/newlib/libgcc.a(_ge_df.o)
                0x0050d4d4                __gedf2
 .text          0x0050d558       0xa0 /home/acer/Andestech/AndeSight133/toolchains/nds32le-elf-V0/libexec/../lib/gcc/nds32le-elf/3.4.4/static/newlib/libgcc.a(_lt_df.o)
                0x0050d574                __ltdf2
 .text          0x0050d5f8       0xf0 /home/acer/Andestech/AndeSight133/toolchains/nds32le-elf-V0/libexec/../lib/gcc/nds32le-elf/3.4.4/static/newlib/libgcc.a(_unpack_df.o)
                0x0050d5f8                __unpack_d
 .text          0x0050d6e8      0x17c /home/acer/Andestech/AndeSight133/toolchains/nds32le-elf-V0/libexec/../lib/gcc/nds32le-elf/3.4.4/static/newlib/libgcc.a(_fpcmp_parts_df.o)
                0x0050d744                __fpcmp_parts_d
 *fill*         0x0050d864        0xc 00000000
 .text          0x0050d870      0x310 /home/acer/Andestech/AndeSight133/toolchains/nds32le-elf-V0/libexec/../nds32le-elf/libc/newlib/usr/lib/libgloss.a(syscalls.o)
                0x0050da28                _argv
                0x0050d9b8                _getpid
                0x0050d8d4                __exit
                0x0050da98                _utime
                0x0050d9b8                __getpid
                0x0050da98                __utime
                0x0050d968                __write
                0x0050d948                __read
                0x0050d99c                __unlink
                0x0050d918                __open
                0x0050da60                __stat
                0x0050db40                isatty
                0x0050d9f0                _fstat
                0x0050db40                _isatty
                0x0050d918                _open
                0x0050d890                _sbrk
                0x0050d9d4                __kill
                0x0050daec                _times
                0x0050da7c                __chmod
                0x0050da60                _stat
                0x0050da0c                __argvlen
                0x0050dad0                __gettimeofday
                0x0050db08                __link
                0x0050da44                _chdir
                0x0050da44                __chdir
                0x0050d980                _lseek
                0x0050da28                __argv
                0x0050dab4                _time
                0x0050db08                _link
                0x0050dab4                __time
                0x0050db24                _rename
                0x0050d980                __lseek
                0x0050da7c                _chmod
                0x0050d99c                _unlink
                0x0050d930                __close
                0x0050d968                _write
                0x0050daec                __times
                0x0050d9d4                _kill
                0x0050db5c                __system
                0x0050dad0                _gettimeofday
                0x0050d948                _read
                0x0050d9f0                __fstat
                0x0050d8d4                _exit
                0x0050db24                __rename
                0x0050da0c                _argvlen
                0x0050db5c                _system
                0x0050d930                _close
 *(.text.*personality*)
 *(.gnu.warning)

.init
 *(.init)

.plt
 *(.plt)

.fini
 *(.fini)
                0x0050db80                PROVIDE (__etext, .)
                0x0050db80                PROVIDE (_etext, .)
                0x0050db80                PROVIDE (etext, .)
                0x00520000                . = ALIGN (0x20000)

.rodata         0x00520000      0x6f8
 *(.rodata .rodata.* .gnu.linkonce.r.*)
 .rodata        0x00520000       0xac hello.o
 .rodata        0x005200ac       0xa8 cmdui.o
 .rodata        0x00520154        0x4 /home/acer/Andestech/AndeSight133/toolchains/nds32le-elf-V0/libexec/../nds32le-elf/libc/newlib/usr/lib/libc.a(impure.o)
                0x00520154                _global_impure_ptr
 .rodata.str1.4
                0x00520158        0x2 /home/acer/Andestech/AndeSight133/toolchains/nds32le-elf-V0/libexec/../nds32le-elf/libc/newlib/usr/lib/libc.a(impure.o)
                                  0x4 (size before relaxing)
 *fill*         0x0052015a        0x2 00
 .rodata        0x0052015c       0x20 /home/acer/Andestech/AndeSight133/toolchains/nds32le-elf-V0/libexec/../nds32le-elf/libc/newlib/usr/lib/libc.a(vfprintf.o)
 .rodata.str1.4
                0x0052017c       0x61 /home/acer/Andestech/AndeSight133/toolchains/nds32le-elf-V0/libexec/../nds32le-elf/libc/newlib/usr/lib/libc.a(vfprintf.o)
                                 0x64 (size before relaxing)
 *fill*         0x005201dd        0x3 00
 .rodata.str1.4
                0x005201e0       0x1e /home/acer/Andestech/AndeSight133/toolchains/nds32le-elf-V0/libexec/../nds32le-elf/libc/newlib/usr/lib/libc.a(wctomb_r.o)
                                 0x20 (size before relaxing)
 *fill*         0x005201fe        0x2 00
 .rodata        0x00520200      0x180 /home/acer/Andestech/AndeSight133/toolchains/nds32le-elf-V0/libexec/../nds32le-elf/libc/newlib/usr/lib/libc.a(ctype_.o)
                0x0052027f                _ctype_
 .rodata.str1.4
                0x00520380       0x10 /home/acer/Andestech/AndeSight133/toolchains/nds32le-elf-V0/libexec/../nds32le-elf/libc/newlib/usr/lib/libc.a(dtoa.o)
                                 0x14 (size before relaxing)
 .rodata.str1.4
                0x00520390        0xc /home/acer/Andestech/AndeSight133/toolchains/nds32le-elf-V0/libexec/../nds32le-elf/libc/newlib/usr/lib/libc.a(locale.o)
                                 0x18 (size before relaxing)
 .rodata        0x0052039c       0x30 /home/acer/Andestech/AndeSight133/toolchains/nds32le-elf-V0/libexec/../nds32le-elf/libc/newlib/usr/lib/libc.a(locale.o)
 *fill*         0x005203cc        0x4 00
 .rodata        0x005203d0      0x128 /home/acer/Andestech/AndeSight133/toolchains/nds32le-elf-V0/libexec/../nds32le-elf/libc/newlib/usr/lib/libc.a(mprec.o)
                0x005203d0                __mprec_tinytens
                0x00520420                __mprec_tens
                0x005203f8                __mprec_bigtens
 .rodata        0x005204f8      0x100 /home/acer/Andestech/AndeSight133/toolchains/nds32le-elf-V0/libexec/../lib/gcc/nds32le-elf/3.4.4/static/newlib/libgcc.a(lib1csrc.o)
 .rodata        0x005205f8      0x100 /home/acer/Andestech/AndeSight133/toolchains/nds32le-elf-V0/libexec/../lib/gcc/nds32le-elf/3.4.4/static/newlib/libgcc.a(_clz.o)
                0x005205f8                __clz_tab

.rodata1
 *(.rodata1)

.sdata2
 *(.sdata2 .sdata2.* .gnu.linkonce.s2.*)

.sbss2
 *(.sbss2 .sbss2.* .gnu.linkonce.sb2.*)

.eh_frame_hdr
 *(.eh_frame_hdr)

.eh_frame
 *(.eh_frame)

.gcc_except_table
 *(.gcc_except_table)
 *(.gcc_except_table.*)
                0x005206f8                . = (ALIGN (0x1000) - ((0x1000 - .) & 0xfff))
                0x00521000                . = (0x1000 DATA_SEGMENT_ALIGN 0x1000)

.eh_frame
 *(.eh_frame)

.gcc_except_table
 *(.gcc_except_table)
 *(.gcc_except_table.*)

.tdata
 *(.tdata .tdata.* .gnu.linkonce.td.*)

.tbss
 *(.tbss .tbss.* .gnu.linkonce.tb.*)
 *(.tcommon)
                0x00521000                . = ALIGN (0x4)
                0x00521000                PROVIDE (__preinit_array_start, .)

.preinit_array
 *(.preinit_array)
                0x00521000                PROVIDE (__preinit_array_end, .)
                0x00521000                PROVIDE (__init_array_start, .)

.init_array
 *(.init_array)
                0x00521000                PROVIDE (__init_array_end, .)
                0x00521000                PROVIDE (__fini_array_start, .)

.fini_array
 *(.fini_array)
                0x00521000                PROVIDE (__fini_array_end, .)

.ctors
 *crtbegin*.o(.ctors)
 *(EXCLUDE_FILE(*crtend*.o) .ctors)
 *(SORT(.ctors.*))
 *(.ctors)

.dtors
 *crtbegin*.o(.dtors)
 *(EXCLUDE_FILE(*crtend*.o) .dtors)
 *(SORT(.dtors.*))
 *(.dtors)

.jcr
 *(.jcr)

.data.rel.ro
 *(.data.rel.ro.local)
 *(.data.rel.ro*)

.dynamic
 *(.dynamic)
                0x00521000                . = (. DATA_SEGMENT_RELRO_END 0x0)

.data           0x00521000     0x5b84
 *(.data .data.* .gnu.linkonce.d.*)
 .data          0x00521000      0xa68 hello.o
 .data          0x00521a68     0x48dc cmdui.o
                0x00521a6c                fLib_CmdTable
                0x00521a68                DefaultStrDelimit
 *fill*         0x00526344        0x4 00
 .data          0x00526348      0x400 /home/acer/Andestech/AndeSight133/toolchains/nds32le-elf-V0/libexec/../nds32le-elf/libc/newlib/usr/lib/libc.a(impure.o)
 .data          0x00526748        0xc /home/acer/Andestech/AndeSight133/toolchains/nds32le-elf-V0/libexec/../nds32le-elf/libc/newlib/usr/lib/libc.a(locale.o)
                0x00526748                __lc_ctype
 .data          0x00526754      0x430 /home/acer/Andestech/AndeSight133/toolchains/nds32le-elf-V0/libexec/../nds32le-elf/libc/newlib/usr/lib/libc.a(mallocr.o)
                0x00526754                __malloc_current_mallinfo
                0x0052677c                __malloc_av_
 *(.gnu.linkonce.d.*personality*)

.sdata_f        0x00526b84        0x3
 .sdata_f       0x00526b84        0x3 /home/acer/Andestech/AndeSight133/toolchains/nds32le-elf-V0/libexec/../lib/gcc/nds32le-elf/3.4.4/static/newlib/libgcc.a(lib1csrc.o)
                0x00526b84                float_detect_tininess
                0x00526b85                float_exception_flags
                0x00526b86                float_rounding_mode

.data1
 *(.data1)
                0x00526b88                . = ALIGN (0x4)

.got
 *(.got.plt)
 *(.got)

.sdata_w        0x00526b88        0x0
                0x00526b88                _SDA_BASE_ = .
                0x00526b88                PROVIDE (__sdata_start, .)
 *(.sdata_w .sdata_w.*)

.sdata_h        0x00526b88       0x40
 *(.sdata_h .sdata_h.*)
 .sdata_h       0x00526b88        0x4 ssp.o
                0x00526b88                TxFIFOLen
 .sdata_h       0x00526b8c        0x4 cmdui.o
                0x00526b8c                DefaultUserSymbolNum
 .sdata_h       0x00526b90        0x4 irq.o
                0x00526b90                fLib_IRQSources
 .sdata_h       0x00526b94        0x4 fiq.o
                0x00526b94                fLib_FIQSources
 .sdata_h       0x00526b98        0x4 /home/acer/Andestech/AndeSight133/toolchains/nds32le-elf-V0/libexec/../nds32le-elf/libc/newlib/usr/lib/libc.a(impure.o)
                0x00526b98                _impure_ptr
 .sdata_h       0x00526b9c        0x4 /home/acer/Andestech/AndeSight133/toolchains/nds32le-elf-V0/libexec/../nds32le-elf/libc/newlib/usr/lib/libc.a(ctype_.o)
                0x00526b9c                __ctype_ptr
 .sdata_h       0x00526ba0       0x14 /home/acer/Andestech/AndeSight133/toolchains/nds32le-elf-V0/libexec/../nds32le-elf/libc/newlib/usr/lib/libc.a(locale.o)
                0x00526bac                __mb_cur_max
                0x00526ba8                __nlocale_changed
                0x00526ba4                __mlocale_changed
                0x00526ba0                _PathLocale
 .sdata_h       0x00526bb4       0x14 /home/acer/Andestech/AndeSight133/toolchains/nds32le-elf-V0/libexec/../nds32le-elf/libc/newlib/usr/lib/libc.a(mallocr.o)
                0x00526bc0                __malloc_top_pad
                0x00526bb8                __malloc_max_sbrked_mem
                0x00526bbc                __malloc_sbrk_base
                0x00526bb4                __malloc_max_total_mem
                0x00526bc4                __malloc_trim_threshold

.sdata_b
 *(.sdata_b .sdata_b.*)
                0x00526bc8                _edata = .
                0x00526bc8                PROVIDE (edata, .)
                0x00526bc8                __bss_start = .

.sbss_b         0x00526bc8        0x0
                0x00526bc8                PROVIDE (__sbss_start, .)
                0x00526bc8                PROVIDE (___sbss_start, .)
 *(.sbss_b .sbss_b.*)
 *(.scommon_b .scommon_b.*)
                0x00526bc8                . = ALIGN (0x2)

.sbss_h         0x00526bc8       0x18
 *(.sbss_h .sbss_h.*)
 .sbss_h        0x00526bc8       0x14 hello.o
 .sbss_h        0x00526bdc        0x4 /home/acer/Andestech/AndeSight133/toolchains/nds32le-elf-V0/libexec/../nds32le-elf/libc/newlib/usr/lib/libc.a(reent.o)
                0x00526bdc                errno
 *(.scommon_h .scommon_h.*)
                0x00526be0                . = ALIGN (0x4)

.sbss_w         0x00526be0        0x0
 *(.sbss_w .sbss_w.*)
 *(.scommon_w .scommon_w.*)
 *(.dynsbss)
 *(.scommon)
                0x00526be0                PROVIDE (__sbss_end, .)
                0x00526be0                PROVIDE (___sbss_end, .)

.bss            0x00526be0     0x2104
 *(.dynbss)
 *(.bss .bss.* .gnu.linkonce.b.*)
 .bss           0x00526be0        0x4 /home/acer/Andestech/AndeSight133/toolchains/nds32le-elf-V0/libexec/../nds32le-elf/libc/newlib/usr/lib/libgloss.a(syscalls.o)
 *(COMMON)
 COMMON         0x00526be4     0x2100 cmdui.o
                0x00526be4                UserSymbolTable
                0x00528ce4                . = ALIGN (0x4)
                0x00528ce4                . = ALIGN (0x4)
                0x00528ce4                _end = .
                0x00528ce4                PROVIDE (end, .)
                0x00528ce4                . = DATA_SEGMENT_END (.)

.stab
 *(.stab)

.stabstr
 *(.stabstr)

.stab.excl
 *(.stab.excl)

.stab.exclstr
 *(.stab.exclstr)

.stab.index
 *(.stab.index)

.stab.indexstr
 *(.stab.indexstr)

.comment        0x00000000      0x522
 *(.comment)
 .comment       0x00000000       0x12 hello.o
 .comment       0x00000012       0x12 ssp.o
 .comment       0x00000024       0x12 cmdui.o
 .comment       0x00000036       0x12 interrupt.o
 .comment       0x00000048       0x12 irq.o
 .comment       0x0000005a       0x12 fiq.o
 .comment       0x0000006c       0x12 /home/acer/Andestech/AndeSight133/toolchains/nds32le-elf-V0/libexec/../nds32le-elf/libc/newlib/usr/lib/libc.a(gets.o)
 .comment       0x0000007e       0x12 /home/acer/Andestech/AndeSight133/toolchains/nds32le-elf-V0/libexec/../nds32le-elf/libc/newlib/usr/lib/libc.a(impure.o)
 .comment       0x00000090       0x12 /home/acer/Andestech/AndeSight133/toolchains/nds32le-elf-V0/libexec/../nds32le-elf/libc/newlib/usr/lib/libc.a(memcpy.o)
 .comment       0x000000a2       0x12 /home/acer/Andestech/AndeSight133/toolchains/nds32le-elf-V0/libexec/../nds32le-elf/libc/newlib/usr/lib/libc.a(printf.o)
 .comment       0x000000b4       0x12 /home/acer/Andestech/AndeSight133/toolchains/nds32le-elf-V0/libexec/../nds32le-elf/libc/newlib/usr/lib/libc.a(strcmp.o)
 .comment       0x000000c6       0x12 /home/acer/Andestech/AndeSight133/toolchains/nds32le-elf-V0/libexec/../nds32le-elf/libc/newlib/usr/lib/libc.a(strcpy.o)
 .comment       0x000000d8       0x12 /home/acer/Andestech/AndeSight133/toolchains/nds32le-elf-V0/libexec/../nds32le-elf/libc/newlib/usr/lib/libc.a(strlen.o)
 .comment       0x000000ea       0x12 /home/acer/Andestech/AndeSight133/toolchains/nds32le-elf-V0/libexec/../nds32le-elf/libc/newlib/usr/lib/libc.a(strncmp.o)
 .comment       0x000000fc       0x12 /home/acer/Andestech/AndeSight133/toolchains/nds32le-elf-V0/libexec/../nds32le-elf/libc/newlib/usr/lib/libc.a(strtok.o)
 .comment       0x0000010e       0x12 /home/acer/Andestech/AndeSight133/toolchains/nds32le-elf-V0/libexec/../nds32le-elf/libc/newlib/usr/lib/libc.a(strtok_r.o)
 .comment       0x00000120       0x12 /home/acer/Andestech/AndeSight133/toolchains/nds32le-elf-V0/libexec/../nds32le-elf/libc/newlib/usr/lib/libc.a(strtoul.o)
 .comment       0x00000132       0x12 /home/acer/Andestech/AndeSight133/toolchains/nds32le-elf-V0/libexec/../nds32le-elf/libc/newlib/usr/lib/libc.a(vfprintf.o)
 .comment       0x00000144       0x12 /home/acer/Andestech/AndeSight133/toolchains/nds32le-elf-V0/libexec/../nds32le-elf/libc/newlib/usr/lib/libc.a(wcrtomb.o)
 .comment       0x00000156       0x12 /home/acer/Andestech/AndeSight133/toolchains/nds32le-elf-V0/libexec/../nds32le-elf/libc/newlib/usr/lib/libc.a(wcsrtombs.o)
 .comment       0x00000168       0x12 /home/acer/Andestech/AndeSight133/toolchains/nds32le-elf-V0/libexec/../nds32le-elf/libc/newlib/usr/lib/libc.a(wctomb_r.o)
 .comment       0x0000017a       0x12 /home/acer/Andestech/AndeSight133/toolchains/nds32le-elf-V0/libexec/../nds32le-elf/libc/newlib/usr/lib/libc.a(wsetup.o)
 .comment       0x0000018c       0x12 /home/acer/Andestech/AndeSight133/toolchains/nds32le-elf-V0/libexec/../nds32le-elf/libc/newlib/usr/lib/libc.a(ctype_.o)
 .comment       0x0000019e       0x12 /home/acer/Andestech/AndeSight133/toolchains/nds32le-elf-V0/libexec/../nds32le-elf/libc/newlib/usr/lib/libc.a(dtoa.o)
 .comment       0x000001b0       0x12 /home/acer/Andestech/AndeSight133/toolchains/nds32le-elf-V0/libexec/../nds32le-elf/libc/newlib/usr/lib/libc.a(fflush.o)
 .comment       0x000001c2       0x12 /home/acer/Andestech/AndeSight133/toolchains/nds32le-elf-V0/libexec/../nds32le-elf/libc/newlib/usr/lib/libc.a(findfp.o)
 .comment       0x000001d4       0x12 /home/acer/Andestech/AndeSight133/toolchains/nds32le-elf-V0/libexec/../nds32le-elf/libc/newlib/usr/lib/libc.a(freer.o)
 .comment       0x000001e6       0x12 /home/acer/Andestech/AndeSight133/toolchains/nds32le-elf-V0/libexec/../nds32le-elf/libc/newlib/usr/lib/libc.a(fvwrite.o)
 .comment       0x000001f8       0x12 /home/acer/Andestech/AndeSight133/toolchains/nds32le-elf-V0/libexec/../nds32le-elf/libc/newlib/usr/lib/libc.a(fwalk.o)
 .comment       0x0000020a       0x12 /home/acer/Andestech/AndeSight133/toolchains/nds32le-elf-V0/libexec/../nds32le-elf/libc/newlib/usr/lib/libc.a(getchar.o)
 .comment       0x0000021c       0x12 /home/acer/Andestech/AndeSight133/toolchains/nds32le-elf-V0/libexec/../nds32le-elf/libc/newlib/usr/lib/libc.a(locale.o)
 .comment       0x0000022e       0x12 /home/acer/Andestech/AndeSight133/toolchains/nds32le-elf-V0/libexec/../nds32le-elf/libc/newlib/usr/lib/libc.a(makebuf.o)
 .comment       0x00000240       0x12 /home/acer/Andestech/AndeSight133/toolchains/nds32le-elf-V0/libexec/../nds32le-elf/libc/newlib/usr/lib/libc.a(mallocr.o)
 .comment       0x00000252       0x12 /home/acer/Andestech/AndeSight133/toolchains/nds32le-elf-V0/libexec/../nds32le-elf/libc/newlib/usr/lib/libc.a(memchr.o)
 .comment       0x00000264       0x12 /home/acer/Andestech/AndeSight133/toolchains/nds32le-elf-V0/libexec/../nds32le-elf/libc/newlib/usr/lib/libc.a(memmove.o)
 .comment       0x00000276       0x12 /home/acer/Andestech/AndeSight133/toolchains/nds32le-elf-V0/libexec/../nds32le-elf/libc/newlib/usr/lib/libc.a(memset.o)
 .comment       0x00000288       0x12 /home/acer/Andestech/AndeSight133/toolchains/nds32le-elf-V0/libexec/../nds32le-elf/libc/newlib/usr/lib/libc.a(mlock.o)
 .comment       0x0000029a       0x12 /home/acer/Andestech/AndeSight133/toolchains/nds32le-elf-V0/libexec/../nds32le-elf/libc/newlib/usr/lib/libc.a(mprec.o)
 .comment       0x000002ac       0x12 /home/acer/Andestech/AndeSight133/toolchains/nds32le-elf-V0/libexec/../nds32le-elf/libc/newlib/usr/lib/libc.a(reallocr.o)
 .comment       0x000002be       0x12 /home/acer/Andestech/AndeSight133/toolchains/nds32le-elf-V0/libexec/../nds32le-elf/libc/newlib/usr/lib/libc.a(rget.o)
 .comment       0x000002d0       0x12 /home/acer/Andestech/AndeSight133/toolchains/nds32le-elf-V0/libexec/../nds32le-elf/libc/newlib/usr/lib/libc.a(s_isinf.o)
 .comment       0x000002e2       0x12 /home/acer/Andestech/AndeSight133/toolchains/nds32le-elf-V0/libexec/../nds32le-elf/libc/newlib/usr/lib/libc.a(s_isnan.o)
 .comment       0x000002f4       0x12 /home/acer/Andestech/AndeSight133/toolchains/nds32le-elf-V0/libexec/../nds32le-elf/libc/newlib/usr/lib/libc.a(sbrkr.o)
 .comment       0x00000306       0x12 /home/acer/Andestech/AndeSight133/toolchains/nds32le-elf-V0/libexec/../nds32le-elf/libc/newlib/usr/lib/libc.a(stdio.o)
 .comment       0x00000318       0x12 /home/acer/Andestech/AndeSight133/toolchains/nds32le-elf-V0/libexec/../nds32le-elf/libc/newlib/usr/lib/libc.a(syssbrk.o)
 .comment       0x0000032a       0x12 /home/acer/Andestech/AndeSight133/toolchains/nds32le-elf-V0/libexec/../nds32le-elf/libc/newlib/usr/lib/libc.a(writer.o)
 .comment       0x0000033c       0x12 /home/acer/Andestech/AndeSight133/toolchains/nds32le-elf-V0/libexec/../nds32le-elf/libc/newlib/usr/lib/libc.a(callocr.o)
 .comment       0x0000034e       0x12 /home/acer/Andestech/AndeSight133/toolchains/nds32le-elf-V0/libexec/../nds32le-elf/libc/newlib/usr/lib/libc.a(closer.o)
 .comment       0x00000360       0x12 /home/acer/Andestech/AndeSight133/toolchains/nds32le-elf-V0/libexec/../nds32le-elf/libc/newlib/usr/lib/libc.a(fclose.o)
 .comment       0x00000372       0x12 /home/acer/Andestech/AndeSight133/toolchains/nds32le-elf-V0/libexec/../nds32le-elf/libc/newlib/usr/lib/libc.a(fstatr.o)
 .comment       0x00000384       0x12 /home/acer/Andestech/AndeSight133/toolchains/nds32le-elf-V0/libexec/../nds32le-elf/libc/newlib/usr/lib/libc.a(lseekr.o)
 .comment       0x00000396       0x12 /home/acer/Andestech/AndeSight133/toolchains/nds32le-elf-V0/libexec/../nds32le-elf/libc/newlib/usr/lib/libc.a(readr.o)
 .comment       0x000003a8       0x12 /home/acer/Andestech/AndeSight133/toolchains/nds32le-elf-V0/libexec/../nds32le-elf/libc/newlib/usr/lib/libc.a(reent.o)
 .comment       0x000003ba       0x12 /home/acer/Andestech/AndeSight133/toolchains/nds32le-elf-V0/libexec/../nds32le-elf/libc/newlib/usr/lib/libc.a(refill.o)
 .comment       0x000003cc       0x12 /home/acer/Andestech/AndeSight133/toolchains/nds32le-elf-V0/libexec/../nds32le-elf/libc/newlib/usr/lib/libc.a(sysclose.o)
 .comment       0x000003de       0x12 /home/acer/Andestech/AndeSight133/toolchains/nds32le-elf-V0/libexec/../nds32le-elf/libc/newlib/usr/lib/libc.a(sysfstat.o)
 .comment       0x000003f0       0x12 /home/acer/Andestech/AndeSight133/toolchains/nds32le-elf-V0/libexec/../nds32le-elf/libc/newlib/usr/lib/libc.a(syslseek.o)
 .comment       0x00000402       0x12 /home/acer/Andestech/AndeSight133/toolchains/nds32le-elf-V0/libexec/../nds32le-elf/libc/newlib/usr/lib/libc.a(sysread.o)
 .comment       0x00000414       0x12 /home/acer/Andestech/AndeSight133/toolchains/nds32le-elf-V0/libexec/../nds32le-elf/libc/newlib/usr/lib/libc.a(syswrite.o)
 .comment       0x00000426       0x12 /home/acer/Andestech/AndeSight133/toolchains/nds32le-elf-V0/libexec/../lib/gcc/nds32le-elf/3.4.4/static/newlib/libgcc.a(_udivsi3.o)
 .comment       0x00000438       0x12 /home/acer/Andestech/AndeSight133/toolchains/nds32le-elf-V0/libexec/../lib/gcc/nds32le-elf/3.4.4/static/newlib/libgcc.a(_umodsi3.o)
 .comment       0x0000044a       0x12 /home/acer/Andestech/AndeSight133/toolchains/nds32le-elf-V0/libexec/../lib/gcc/nds32le-elf/3.4.4/static/newlib/libgcc.a(lib1csrc.o)
 .comment       0x0000045c       0x12 /home/acer/Andestech/AndeSight133/toolchains/nds32le-elf-V0/libexec/../lib/gcc/nds32le-elf/3.4.4/static/newlib/libgcc.a(_negdi2.o)
 .comment       0x0000046e       0x12 /home/acer/Andestech/AndeSight133/toolchains/nds32le-elf-V0/libexec/../lib/gcc/nds32le-elf/3.4.4/static/newlib/libgcc.a(_udivdi3.o)
 .comment       0x00000480       0x12 /home/acer/Andestech/AndeSight133/toolchains/nds32le-elf-V0/libexec/../lib/gcc/nds32le-elf/3.4.4/static/newlib/libgcc.a(_umoddi3.o)
 .comment       0x00000492       0x12 /home/acer/Andestech/AndeSight133/toolchains/nds32le-elf-V0/libexec/../lib/gcc/nds32le-elf/3.4.4/static/newlib/libgcc.a(_eq_df.o)
 .comment       0x000004a4       0x12 /home/acer/Andestech/AndeSight133/toolchains/nds32le-elf-V0/libexec/../lib/gcc/nds32le-elf/3.4.4/static/newlib/libgcc.a(_ne_df.o)
 .comment       0x000004b6       0x12 /home/acer/Andestech/AndeSight133/toolchains/nds32le-elf-V0/libexec/../lib/gcc/nds32le-elf/3.4.4/static/newlib/libgcc.a(_gt_df.o)
 .comment       0x000004c8       0x12 /home/acer/Andestech/AndeSight133/toolchains/nds32le-elf-V0/libexec/../lib/gcc/nds32le-elf/3.4.4/static/newlib/libgcc.a(_ge_df.o)
 .comment       0x000004da       0x12 /home/acer/Andestech/AndeSight133/toolchains/nds32le-elf-V0/libexec/../lib/gcc/nds32le-elf/3.4.4/static/newlib/libgcc.a(_lt_df.o)
 .comment       0x000004ec       0x12 /home/acer/Andestech/AndeSight133/toolchains/nds32le-elf-V0/libexec/../lib/gcc/nds32le-elf/3.4.4/static/newlib/libgcc.a(_clz.o)
 .comment       0x000004fe       0x12 /home/acer/Andestech/AndeSight133/toolchains/nds32le-elf-V0/libexec/../lib/gcc/nds32le-elf/3.4.4/static/newlib/libgcc.a(_unpack_df.o)
 .comment       0x00000510       0x12 /home/acer/Andestech/AndeSight133/toolchains/nds32le-elf-V0/libexec/../lib/gcc/nds32le-elf/3.4.4/static/newlib/libgcc.a(_fpcmp_parts_df.o)

.debug
 *(.debug)

.line
 *(.line)

.debug_srcinfo
 *(.debug_srcinfo)

.debug_sfnames
 *(.debug_sfnames)

.debug_aranges  0x00000000       0xe0
 *(.debug_aranges)
 .debug_aranges
                0x00000000       0x20 hello.o
 .debug_aranges
                0x00000020       0x20 ssp.o
 .debug_aranges
                0x00000040       0x20 cmdui.o
 .debug_aranges
                0x00000060       0x20 interrupt.o
 .debug_aranges
                0x00000080       0x20 irq.o
 .debug_aranges
                0x000000a0       0x20 fiq.o
 .debug_aranges
                0x000000c0       0x20 boot.o

.debug_pubnames
                0x00000000      0x44a
 *(.debug_pubnames)
 .debug_pubnames
                0x00000000       0x35 hello.o
 .debug_pubnames
                0x00000035      0x138 ssp.o
 .debug_pubnames
                0x0000016d      0x224 cmdui.o
 .debug_pubnames
                0x00000391       0x39 interrupt.o
 .debug_pubnames
                0x000003ca       0x40 irq.o
 .debug_pubnames
                0x0000040a       0x40 fiq.o

.debug_info     0x00000000     0x1c56
 *(.debug_info .gnu.linkonce.wi.*)
 .debug_info    0x00000000      0x593 hello.o
 .debug_info    0x00000593      0x4af ssp.o
 .debug_info    0x00000a42      0xceb cmdui.o
 .debug_info    0x0000172d      0x19f interrupt.o
 .debug_info    0x000018cc      0x1a1 irq.o
 .debug_info    0x00001a6d      0x1a1 fiq.o
 .debug_info    0x00001c0e       0x48 boot.o

.debug_abbrev   0x00000000      0x4de
 *(.debug_abbrev)
 .debug_abbrev  0x00000000      0x110 hello.o
 .debug_abbrev  0x00000110       0xc0 ssp.o
 .debug_abbrev  0x000001d0      0x172 cmdui.o
 .debug_abbrev  0x00000342       0x6e interrupt.o
 .debug_abbrev  0x000003b0       0x8d irq.o
 .debug_abbrev  0x0000043d       0x8d fiq.o
 .debug_abbrev  0x000004ca       0x14 boot.o

.debug_line     0x00000000      0x533
 *(.debug_line)
 .debug_line    0x00000000       0xcd hello.o
 .debug_line    0x000000cd       0xa8 ssp.o
 .debug_line    0x00000175      0x28a cmdui.o
 .debug_line    0x000003ff       0x68 interrupt.o
 .debug_line    0x00000467       0x45 irq.o
 .debug_line    0x000004ac       0x45 fiq.o
 .debug_line    0x000004f1       0x42 boot.o

.debug_frame    0x00000000      0x2f0
 *(.debug_frame)
 .debug_frame   0x00000000       0x40 hello.o
 .debug_frame   0x00000040       0xc0 ssp.o
 .debug_frame   0x00000100      0x160 cmdui.o
 .debug_frame   0x00000260       0x30 interrupt.o
 .debug_frame   0x00000290       0x30 irq.o
 .debug_frame   0x000002c0       0x30 fiq.o

.debug_str      0x00000000       0x95
 *(.debug_str)
 .debug_str     0x00000000       0x1e hello.o
 .debug_str     0x0000001e       0x1a ssp.o
 .debug_str     0x00000038       0x36 cmdui.o
 .debug_str     0x0000006e        0xd interrupt.o
 .debug_str     0x0000007b        0xd irq.o
 .debug_str     0x00000088        0xd fiq.o

.debug_loc
 *(.debug_loc)

.debug_macinfo
 *(.debug_macinfo)

.debug_weaknames
 *(.debug_weaknames)

.debug_funcnames
 *(.debug_funcnames)

.debug_typenames
 *(.debug_typenames)

.debug_varnames
 *(.debug_varnames)
                0x00540000                PROVIDE (_stack, 0x540000)

/DISCARD/
 *(.note.GNU-stack)
LOAD /home/acer/Andestech/AndeSight133/toolchains/nds32le-elf-V0/libexec/../lib/gcc/nds32le-elf/3.4.4/static/newlib/libgcc.a
LOAD /home/acer/Andestech/AndeSight133/toolchains/nds32le-elf-V0/libexec/../nds32le-elf/libc/newlib/usr/lib/libc.a
LOAD /home/acer/Andestech/AndeSight133/toolchains/nds32le-elf-V0/libexec/../lib/gcc/nds32le-elf/3.4.4/static/newlib/libgcc.a
START GROUP
LOAD /home/acer/Andestech/AndeSight133/toolchains/nds32le-elf-V0/libexec/../lib/gcc/nds32le-elf/3.4.4/static/newlib/libgcc.a
LOAD /home/acer/Andestech/AndeSight133/toolchains/nds32le-elf-V0/libexec/../nds32le-elf/libc/newlib/usr/lib/libandestar32_generic.a
LOAD /home/acer/Andestech/AndeSight133/toolchains/nds32le-elf-V0/libexec/../nds32le-elf/libc/newlib/usr/lib/libc.a
LOAD /home/acer/Andestech/AndeSight133/toolchains/nds32le-elf-V0/libexec/../nds32le-elf/libc/newlib/usr/lib/libm.a
LOAD /home/acer/Andestech/AndeSight133/toolchains/nds32le-elf-V0/libexec/../nds32le-elf/libc/newlib/usr/lib/libgloss.a
END GROUP
OUTPUT(hello.dbg elf32-nds32)

.mdebug.abi_nds32
                0x00000000        0x0
